S02000006F70656E626C745F6F6C696D65785F73746D3332683130332E737265630F
S3150800000000500020BD2200080D2300080D2300081B
S315080000100D2300080D2300080D230008000000002A
S315080000200000000000000000000000000D2300088A
S315080000300D230008000000000D2300080D2300080A
S315080000400D2300080D2300080D2300080D230008C2
S315080000500D2300080D2300080D2300080D230008B2
S315080000600D2300080D2300080D2300080D230008A2
S315080000700D2300080D2300080D2300080D23000892
S315080000800D2300080D2300080D2300080D23000882
S315080000900D2300080D2300080D2300080D23000872
S315080000A00D2300080D2300080D2300080D23000862
S315080000B00D2300080D2300080D2300080D23000852
S315080000C00D2300080D2300080D2300080D23000842
S315080000D00D2300080D2300080D2300080D23000832
S315080000E00D2300080D2300080D230008000000005A
S315080000F000000000000000000000000000000000F2
S3110800010000000000000000005FF808F195
S3150800010C10B5054C237833B9044B13B10448AFF337
S3150800011C00800123237010BDF000002000000000B1
S3150800012CE025000808B5034B1BB103490348AFF398
S3150800013C008008BD00000000F4000020E02500083F
S3150800014C72B6704762B6704708B5FFF7F9FF08BD77
S3150800015C10B500F0B3FA00B910BD00F099FF0028ED
S3150800016CFAD000F043FD00F0BDFA00F0ABFA20F02F
S3150800017C604020F07F00044B186000F0A3FA446836
S3150800018CFFF7E0FFA047E7E708ED00E070B508E0E9
S3150800019C461C4D1C0B78037000F057FD304629465B
S315080001AC2246531E9CB2002AF2D170BD044B054A56
S315080001BC5A6002F188325A603422DA60704700BFFE
S315080001CC0020024023016745024A136943F0800365
S315080001DC136170470020024038B50546002401E03B
S315080001EC0134E4B20D2C15D800F02FFD04EB4402B3
S315080001FC9300094AD358AB42F2D804EB4402910057
S3150800020C054A0A44526813449D42E9D2024B0B44F0
S3150800021C187A38BDFF2038BDF825000838B50546CC
S3150800022C00240D2C10D800F010FD04EB44039A00A2
S3150800023C074B13441B7AAB4202D00134E4B2F0E705
S3150800024C1346034AD05838BD4FF0FF3038BD00BFAF
S3150800025CF825000838B5054600240D2C10D800F0F2
S3150800026CF4FC04EB44039A00064B13441B7AAB428A
S3150800027C02D00134E4B2F0E7024B1344586838BD97
S3150800028C002038BDF825000808B5C1F3080353B992
S3150800029C0368994209D040F8041B4FF40072FFF723
S315080002AC75FF012008BD002008BD012008BD00000F
S315080002BC2DE9F84F81460068FFF78EFFFF2856D0C8
S315080002CCFFF774FF2B4BDB6813F0010F08D1294A93
S315080002DC136943F00103136100254FF0010A09E085
S315080002ECFFF772FF4FF0000A3EE058F807309E42BF
S315080002FC31D101357F2D30D8D9F80080AF0008EB05
S3150800030C070B09EB07035E68B3B228F8253000F033
S3150800031C11FA441D174BDB6813F0010F07D000F0D8
S3150800032C94FC00F007FA8442F4D24FF0000A330C1E
S3150800033CABF8023000F0FEF9441D0E4BDB6813F0E7
S3150800034C010FD2D000F081FC00F0F4F98442F4D20B
S3150800035C4FF0000AC9E74FF0000A064A136923F062
S3150800036C01031361FFF730FF5046BDE8F88F4FF0D5
S3150800037C000AF9E70020024038B50D460B4B9842A7
S3150800038C08D004460A4B994206D0FFF791FF20B9CC
S3150800039C002407E0074C00E0044C29462046FFF7EA
S315080003AC73FF08B1204638BD0024FBE71003002074
S315080003BC004000080C0100202DE9F04106460C46C9
S315080003CC17461D4621F4FF7828F001080368B3F197
S315080003DCFF3F0DD03368984505D041463046FFF7A8
S315080003ECCBFF064628B33368E41A344404340CE0CD
S315080003FC4146FFF749FF03460028EBD116E017F8EC
S3150800040C013B04F8013B013D0FD000F01EFC331DE7
S3150800041CE31AB3F5007FF2D308F500713046FFF7FF
S3150800042CABFF064638B1041DE9E701231846BDE8BB
S3150800043CF0810023FAE70023F8E700002DE9F041E4
S3150800044C884251D8012853D90F2901D900264CE0E6
S3150800045C0D460446FFF7AAFE264BDB6813F0010F80
S3150800046C19D1244A136943F0020313612046FFF796
S3150800047CD5FE80462846FFF7D1FE07462846FFF7E5
S3150800048CE9FE0744013FA7EB08070137C7F38F2797
S3150800049C0126002505E0FFF797FE002625E0013525
S315080004ACADB2BD4218D208EB8522124B5A611A69B5
S315080004BC42F040021A6100F03DF900F164040D4B5C
S315080004CCDB6813F0010FEAD000F0BFFB00F032F93D
S315080004DC8442F4D20026E2E7064A136923F00203A3
S315080004EC1361FFF771FE00E000263046BDE8F08187
S315080004FC0026FAE7002002404FF0FF33024A136049
S3150800050C024A1360704700BF0C010020100300203C
S3150800051C70B54B1E154C241AA34201D9002070BD88
S3150800052C16460D460446FFF757FEFF281AD028191B
S3150800053C0138FFF751FEFF2816D024F4FF7323F079
S3150800054C01030B4A934206D02B46324621460948EC
S3150800055CFFF732FF70BD2B46324621460648FFF799
S3150800056C2BFF70BD002070BD002070BDFFFF010879
S3150800057C004000080C010020100300204A1E0E4BF8
S3150800058C1B1A9A4201D90020704770B50C460546CD
S3150800059CFFF722FE064660190138FFF71DFEFF2EEF
S315080005AC06D0FF2806D001463046FFF747FF70BD38
S315080005BC002070BD002070BDFFFF0108104B1B68A2
S315080005CCB3F1FF3F1AD000B583B00D4A5368916852
S315080005DC0B44D1680B4411690B4451690B4491695E
S315080005EC0B44D26913445B4202AA42F8043D042127
S315080005FC0448FFF78DFF03B05DF804FB0120704734
S3150800060C100300200C4100080D4B1B680D4A12689C
S3150800061C13440D4A126813440C4A126813440C4AC4
S3150800062C126813440B4A126813440B4A1268134493
S3150800063C0A4A1268D34201D000207047012070473D
S3150800064C0040000804400008084000080C40000858
S3150800065C1040000814400008184000080C41000817
S3150800066C08B50C4B1B68B3F1FF3F04D00948FFF7DC
S3150800067C1FFE034650B1084B1B68B3F1FF3F07D06A
S3150800068C0548FFF715FE034600B10123184608BDB9
S3150800069C0123FBE7100300200C01002000487047DB
S315080006AC0040000808B5FFF727FF08BD08B5FFF797
S315080006BC2FFF08BD08B5FFF761FF08BD08B5FFF7A2
S315080006CCA3FF08BD08B5FFF7E9FF08BD08B5FFF796
S315080006DC75FF034608B9184608BDFFF7C1FF034660
S315080006ECF9E700000022014B1A60704710E000E0A1
S315080006FC08B5FFF7F7FF054B054A5A6000229A60C2
S3150800070C05211960034B1A6008BD00BF10E000E014
S3150800071C3F19010014050020044B1B6813F4803F95
S3150800072C03D0034A136801331360704710E000E0E6
S3150800073C1405002008B5FFF7EFFF014B186808BD34
S3150800074C140500200023934216D230B40BE037343C
S3150800075C01F8134000015C00013400250D550133E6
S3150800076CDBB2934206D2040F092CF0D8303401F8C8
S3150800077C1340EFE730BC704770470000094B03F194
S3150800078C1801002232B19A7400225A61054A064BA6
S3150800079C1A6070479A745961183318310132D2B2FB
S315080007ACF0E700BF98050020C80500200A4B1B6817
S315080007BC7BB110B45C69084A146019749860D860E7
S315080007CC00225A741860013908445860987C10BC89
S315080007DC7047FF20704700BFC805002038B504468F
S315080007EC0D46012804D94FF4FA71124800F090F915
S315080007FC62002244D100104B0B445A7C1B7C9A4253
S3150800080C13D00D4B0B44DA6815705A7C01325A74A6
S3150800081CDA680132DA605B689A4208D9064A0846F1
S3150800082C51580244D160012038BD002038BD012042
S3150800083C38BD00BFA02600089805002008B501465B
S3150800084C024B1878FFF7CAFF08BD00BFCC0500207D
S3150800085C38B504460D46012804D940F2162113482A
S3150800086C00F056F904EB4403DA00114B13445B7C95
S3150800087CBBB162002244D1000D4B0B449A68127826
S3150800088C2A705A7C013A5A749A6801329A605B68E3
S3150800089C9A4208D9064A08465158024491600120E2
S315080008AC38BD002038BD012038BD00BFA026000881
S315080008BC9805002008B50146024B1878FFF7C8FFC3
S315080008CC08BD00BF1006002010B50446012804D93F
S315080008DC40F23621044800F01BF904EB4404E2000C
S315080008EC024B1344587C10BDA0260008980500201E
S315080008FC38B5FFF743FF0C4C4021601CFFF756FF39
S3150800090C20700A4D4021681CFFF750FF2870237889
S3150800091CFF2B04D0FF2802D001F060F938BD7321F3
S3150800092C034800F0F5F8F7E7CC0500201006002080
S3150800093CA026000808B5002000F084FB08BD0000BE
S3150800094C70B506460D463F290AD82846FFF776FFA6
S3150800095C012803D096210E4800F0DAF8002406E0A8
S3150800096C92210B4800F0D4F8EFE70134A4B2ABB2ED
S3150800097C9C420BD200F069F9305DFFF75FFF012846
S3150800098CF3D09F21024800F0C3F8EEE770BD00BF14
S3150800099CA026000870B506460D4601F0C7FC1C4B90
S315080009AC1C789CB91B48FFF785FF012801D0204607
S315080009BC70BD184B1B78013BDBB23E2BF7D80122D6
S315080009CC134B1A700022144B1A70F0E7124B1B7853
S315080009DC013310481844FFF76DFF0446012801D06F
S315080009EC0024E4E70C4B1A780132D2B21A70094B80
S315080009FC1B789A4201D00024D9E708493046FFF7FC
S31508000A0CC5FB0022024B1A70034B1B782B70CEE7E2
S31508000A1C9406002054060020950600205506002052
S31508000A2C30B583B0184B1878FFF74EFF48B3054618
S31508000A3C402800D94025002405E09DF80720134BD3
S31508000A4C1A550134E4B2A5420DD90DF107010E4B26
S31508000A5C1878FFF7FDFE0128EFD040F245110C4837
S31508000A6C00F056F8E9E7ADB22A464FF4807107480C
S31508000A7C01F002FA2946012001F00EFB012001F0D3
S31508000A8C70FA03B030BD00BFCC0500205805002015
S31508000A9CA026000838B50E49012001F053FB85B293
S31508000AAC002401E00134A4B2AC420DD2084B195D06
S31508000ABC084B1878FFF792FE0128F3D04FF4B5715E
S31508000ACC054800F025F8EDE7012001F05DFA38BD80
S31508000ADC1805002010060020A026000838B50A4B79
S31508000AEC186804331C6804331B68C01800D138BD59
S31508000AFC064D08222946FFF725FE042205F11001AA
S31508000B0C2046FFF71FFEF2E7E8F7FF1F0600002056
S31508000B1C08B500F09AF8FCE708B500F091F801283A
S31508000B2C03D0094B1B78012B00D008BDFFF702FE3A
S31508000B3C064B1B6803F5FA639842F6D30022024B60
S31508000B4C1A70FFF705FBF0E79606002098060020BA
S31508000B5C08B50122044B1A70FFF7ECFD034B18601D
S31508000B6CFFF7DAFF08BD00BF96060020980600209E
S31508000B7C08B5FFF7E9FA00F067F8FFF7B9FDFFF7D4
S31508000B8C91FD00F00DF8FFF7E3FF08BD08B500F07E
S31508000B9C5CF8FFF7C1FD00F00FF8FFF7BDFF08BDC5
S31508000BAC08B500F0BDF9FFF7A3FE0222014B1A7037
S31508000BBC08BD00BF0000002000B583B00DF1070189
S31508000BCC0848FFF7E7FE012802D003B05DF804FBDE
S31508000BDC0222054B1A709DF80710024800F0C0F95E
S31508000BECF3E700BF9C0600200000002008B5FFF7BD
S31508000BFCA1FE08BD08B5054B1B78022B02D000F0E8
S31508000C0CA7F908BDC9B2FFF79BFEF8E7000000205C
S31508000C1C044B1B78012B03D9032B01D03F207047BB
S31508000C2C0020704700000020044B1B78012B03D9C9
S31508000C3C032B01D03F20704700207047000000208E
S31508000C4C08B500F07BF908BD704770470022014BC8
S31508000C5C5A707047DC060020034BFE22DA701871B6
S31508000C6C0222A3F844207047DC06002010B5054C78
S31508000C7C00232370FFF7EAFFFF23E3700123A4F890
S31508000C8C443010BDDC060020064BFF22DA70002229
S31508000C9C1A71597859719A71DA711A720622A3F86F
S31508000CAC44207047DC06002008B50020FFF7D4FF67
S31508000CBC08BD0000074BFF22DA70074A9A64002227
S31508000CCC1A715A719A710722C3F807200822A3F8D9
S31508000CDC44207047DC060020C8260008044BFF2277
S31508000CECDA7042689A640122A3F84420704700BF60
S31508000CFCDC06002008B53120FFF7AEFF08BD000062
S31508000D0C38B5084CFF23E370002525716571FFF78C
S31508000D1C7FFFA071E571257265720723A4F844302C
S31508000D2C38BD00BFDC06002038B5FFF78FFF0E4C28
S31508000D3C01252570FF23E3701023237100236371AB
S31508000D4CFFF766FFA071FFF76FFFE071FFF76CFF07
S31508000D5CC0F3072020726572A5720823A4F84430E4
S31508000D6CFFF7A0FC38BD00BFDC06002038B50546E9
S31508000D7C4478FFF74DFF0138844210DC0A4C6A7838
S31508000D8CA16C201DFFF702FAFF23E3706A78A36CA7
S31508000D9C1344A3646B780133A4F8443038BD22207D
S31508000DACFFF75AFF38BD00BFDC06002038B50446ED
S31508000DBC4578FFF72DFF0138854211DC61680A4D2D
S31508000DCCA9646278281DFFF7E1F9FF23EB706278B6
S31508000DDCAB6C1344AB6463780133A5F8443038BD67
S31508000DEC2220FFF739FF38BDDC060020F8B505468A
S31508000DFC1746002406E015F8013B1C44E4B2FFF73D
S31508000E0C24FF31464E1E0029F5D13C600120F8BD61
S31508000E1C10B5084CFF23E370E21D4168A06CFFF780
S31508000E2CE5FF207100236371A3710823A4F84430ED
S31508000E3C10BD00BFDC06002038B505460D4B9C6C72
S31508000E4CFFF7E6FE6A1C411E2046FFF72FFC60B131
S31508000E5C084CFF23E370FFF7DBFE0138A36C034451
S31508000E6CA3640123A4F8443038BD3120FFF7F4FEFF
S31508000E7C38BD00BFDC06002038B504464578FFF7B8
S31508000E8CC7FE023885420EDC114BFF22DA700122AE
S31508000E9CA3F84420617851B9FFF718FC90B93120B2
S31508000EACFFF7DAFE38BD2220FFF7D6FE38BDA21CA6
S31508000EBC074B986CFFF7FAFB28B16178044A936CD8
S31508000ECC0B44936438BD3120FFF7C6FE38BD00BF0E
S31508000EDCDC06002008B54168074B986CFFF7EAFB5F
S31508000EEC30B1054BFF22DA700122A3F8442008BD65
S31508000EFC3120FFF7B1FE08BDDC06002008B5FFF768
S31508000F0C27F9034BFF22DA700122A3F8442008BD07
S31508000F1CDC06002008B589B2FFF76CFE08BD000098
S31508000F2C054B00221A709A6483F84220A3F84420D1
S31508000F3C9A705A70704700BFDC060020034B1B786A
S31508000F4C0BB1012070470020704700BFDC0600205B
S31508000F5C0022024B83F84220704700BFDC060020B3
S31508000F6C08B50378FF2B04D0354A1278012A14D019
S31508000F7C08BDFFF7D9FE324B93F84230012B5AD0F5
S31508000F8C2F4BB3F944100029F2DD1846012380F8DB
S31508000F9C42300330FFF7BEFFEAE7C93B352B46D88C
S31508000FACDFE803F03345454245453F363C39454570
S31508000FBC45454545454545454545454545454545C7
S31508000FCC4545454545454545454545454545241EFF
S31508000FDC1B2145454527452A2D30FFF7C7FECAE78D
S31508000FECFFF7E4FEC7E7FFF779FEC4E7FFF710FF44
S31508000FFCC1E7FFF75FFEBEE7FFF756FEBBE7FFF755
S3150800100C43FEB8E7FFF732FEB5E7FFF715FFB2E781
S3150800101CFFF732FFAFE7FFF773FEACE7FFF75AFFB0
S3150800102CA9E7FFF76BFFA6E7FFF764FEA3E7202007
S3150800103CFFF712FE9FE71020FFF70EFEA0E700BF92
S3150800104CDC0600200F4B1B7883B90F4A936943F0D3
S3150800105C100393610D4B5A6822F470425A605A6811
S3150800106C42F4E0425A600122064B1A70012804D059
S3150800107C4FF40062054B1A6170474FF40062034B3C
S3150800108C5A617047280700200010024000100140E2
S3150800109C044B9B6813F0010F01D001207047002008
S315080010AC704700BF0008014082B0002301930093EB
S315080010BC2C4A136843F4803313602A4B1B6803F4D9
S315080010CC00330093019B01330193009B1BB9019BD1
S315080010DCB3F5A06FF1D1234B1B6813F4003F06D070
S315080010EC01230093009B012B04D002B07047002308
S315080010FC0093F7E71C4B1A6842F010021A601A683C
S3150800110C22F003021A601A6842F002021A60A3F56A
S3150800111C80535A685A605A685A605A6842F4806210
S3150800112C5A605A6822F47C125A605A6842F4E812D9
S3150800113C5A601A6842F080721A600A4B1B6813F0E0
S3150800114C007FFAD0074B5A6822F003025A605A6895
S3150800115C42F002025A60034B5B6803F00C03082B3F
S3150800116CF9D1C2E7001002400020024008B5FFF78B
S3150800117C9BFF08BD08B5104B1A6842F001021A60AD
S3150800118C59680E4A0A405A601A6822F0847222F488
S3150800119C80321A601A6822F480221A605A6822F47D
S315080011ACFE025A604FF41F029A60FFF7DFFF4FF0FA
S315080011BC0062034B9A6008BD001002400000FFF85D
S315080011CC00ED00E008B538B1064B1B681B6898475C
S315080011DC054B18680A3008BD034B1B6801221A8296
S315080011EC08BD00BF5C0700206007002008B538B1B1
S315080011FC064B1B689B689847054B18680C3008BD4E
S3150800120C034B1B6801221A8208BD00BF5C0700202D
S3150800121C6007002008B5E8B10022294B1A80294B33
S3150800122C1A68137813F07F031FD1537A13F0200F23
S3150800123C02D00221224A117013F0400F0FD0204A17
S3150800124C137843F0010313701F4B1B681B699847EF
S3150800125C1B4808BD1B4B1B6802221A8208BD184A7C
S3150800126C137823F001031370EEE7012B24D0022B1D
S3150800127C24D1527902F00F0312F0800F0ED19B0085
S3150800128C03F1804303F5B8431B6803F44053B3F5E5
S3150800129C805FD9D101220A4B1A70D5E79B0003F15E
S315080012AC804303F5B8431B6803F03003102BCBD1EE
S315080012BC0122034B1A70C7E7014808BD002008BD78
S315080012CC30070020600700205C070020F8B5254B86
S315080012DC1D682C8A2B7A0CB9042B28D0AB8A9C4215
S315080012EC3DD804269C4200D31C46AB69A4B22046C2
S315080012FC98470746002000F0B3FE224601463846BA
S3150800130C00F0BAFD2146002000F0C6FE2B8A1B1BF6
S3150800131C2B826B8A1C446C823022134B1A804FF436
S3150800132C4052124B1A800F4B1B681E72F8BD104B9D
S3150800133C1B78012B04D010220B4B1A800726F2E7D8
S3150800134C0C4B1A6892B20C4B13445B0000221A60C1
S3150800135C3021054B1980064B1A700426E3E7022642
S3150800136CC0E700BF6007002068070020660700205A
S3150800137C29070020505C00400230002010B582B0CE
S3150800138C804B1A685378062B32D03BB9518829B949
S3150800139C516821F47F41B1F5003F42D0082B7FD02C
S315080013AC0A2B00F083800023002B00F0AD80754AD1
S315080013BC126800245482936120469847714B1B6827
S315080013CC1A8A4FF6FF718A4200F0AE80022C00F0A2
S315080013DCAE80002A00F0AB8093F900100029C0F209
S315080013ECAA8003221A724FF44052674B1A80A0E067
S315080013FC137813F07F0F75D19378012B05D0022B38
S3150800140C07D0032B09D00023CEE7604B1B68DB699A
S3150800141CCAE75E4B1B681B6AC6E75C4B1B685B6AB4
S3150800142CC2E7137813F07F0302D1918800295BD0A9
S3150800143C012B03D0022B10D00023B5E7534B1B68A6
S3150800144C9B6900215079984700284FD14D4B1B6852
S3150800145C9B7A002BA8D04E4BA6E7537903F00F02C4
S3150800146C03F0700013F0800F11D1930003F1804341
S3150800147C03F5B8431B6803F44053464909788A4276
S3150800148C36D2002836D1002B8ED0414B8CE79300F0
S3150800149C03F1804303F5B8431B6803F03003ECE70C
S315080014AC137813F07F0F27D000237DE7137803F00A
S315080014BC7F03012B01D0002376E7937AF3B1538887
S315080014CCF3B9536823F47F43B3F5803F01D0002367
S315080014DC6AE72E4B1B689B6900215079984788B19F
S315080014EC002361E700235FE7294B5DE700235BE7F1
S315080014FC002359E7002357E7274B55E7002353E703
S3150800150C002351E7254B4FE7204B1B681B691D4AE7
S3150800151C126850789847044603287FF44FAF194B46
S3150800152C1B6809221A7204E009221A7201E00822C1
S3150800153C1A7202B010BDD98801910198824209D954
S3150800154C019A1A82114A126892F82C209A82FFF78D
S3150800155CBDFEEEE78A42F5D20C49096891F82C10C3
S3150800156C88B2824203D200210D4A1170EAE792FB37
S3150800157CF1F001FB1022002AE4D10121084A11706E
S3150800158CE0E700BF60070020660700203807002048
S3150800159C21120008A0000020D1110008F91100083A
S315080015AC2907002070B5244B1C68258AA369B3B19A
S315080015BCADB1A18A8D4200D30D46ADB228469847E7
S315080015CC0646238A5B1B2382638A2B44638200208C
S315080015DC00F054FD2A460146304600F063FC238A87
S315080015ECA3B9238AA28A93421CD203BB124B1B684B
S315080015FC06221A72114B1A6892B2114B13445B00ED
S3150800160C00221A6030220F4B1A8070BD4FF44052DC
S3150800161C0D4B1A800021084600F03EFD3022094B7E
S3150800162C1A80DEE7044B1B6803221A7270BD024B44
S3150800163C1B6805221A7270BD60070020505C0040BA
S3150800164C02300020680700206607002008B50C4BFE
S3150800165C1B68DA780B4949788A4201D9022008BDF9
S3150800166C997809B1022008BD998809B1022008BDEC
S3150800167C9A72054B1B685B689847002008BD00BF2B
S3150800168C60070020A00000205C07002038B5124B2C
S3150800169C1B689A69114D2B68D978587990472B682D
S315080016AC9A7A12B90224204638BD044608B1022497
S315080016BCF9E71A790AB10224F5E79B780BB10224EB
S315080016CCF1E7074B1B68DB6898472B685A79DA727F
S315080016DCDA781A73E7E700BF38070020600700209E
S315080016EC5C070020434B1A68137813F07F0303D06A
S315080016FC022B07D002207047537A23F0200353722B
S3150800170C0020704753880BB10220704713790BB130
S3150800171C0220704710B5537923F080005BB2002B7A
S3150800172C0DDB810001F1804101F5B841096801F42E
S3150800173C4051314C2478A0420AD3022010BD8100B6
S3150800174C01F1804101F5B841096801F03001F0E773
S3150800175C09B9022010BD927A0AB9022010BD002BD5
S3150800176C10DB840004F1804404F5B844236803F4C0
S3150800177C4053B3F5805F18D0204B1B685B699847BC
S3150800178C002010BD830003F1804303F5B8431B68A2
S3150800179C03F03003102BEFD1C4B2204600F02CFC1A
S315080017AC3021204600F0A5FBE6E790B9144B93F8D8
S315080017BC2C1000F07FFC23689BB223F4804323F0A3
S315080017CC700383F4405343F4004343F080032360CF
S315080017DCD2E700F0FDFB23689BB223F4804323F089
S315080017EC700383F4405343F4004343F080032360AF
S315080017FCC2E700BF60070020A00000205C0700209D
S3150800180C7000002010B52B4B1868437923F0800123
S3150800181C5BB2002B0DDB8A0002F1804202F5B8425E
S3150800182C126802F44052244C2478A1420AD30220AE
S3150800183C10BD8A0002F1804202F5B842126802F025
S3150800184C3002F0E744880CB1022010BD0AB9022018
S3150800185C10BD827A0AB9022010BD002B17DB8B004B
S3150800186C03F1804303F5B8431A6892B222F4804216
S3150800187C22F0700282F4805242F4004242F0800256
S3150800188C1A600E4B1B689B699847002010BD8A008E
S3150800189C02F1804202F5B84213689BB223F4E04386
S315080018AC23F0400383F0100343F4004343F0800312
S315080018BC1360E6E760070020A00000205C07002004
S315080018CC08B5064B1A68537A43F020035372044B37
S315080018DC1B68DB699847002008BD00BF600700201D
S315080018EC5C07002010B5404B1A685478137813F02F
S315080018FC7F0338D1092C07D0052C08D0032C15D01A
S3150800190C012C1FD0022033E0FFF7A0FE30E092F93D
S3150800191C0330002B5DDB9378002B5CD19388002B6E
S3150800192C5BD1937A002B5AD1002021E0D378012B76
S3150800193C01D002201CE093880BB1022018E0FFF7B7
S3150800194CBFFF15E0D378012B01D0022010E0938855
S3150800195C002B33D1537A13F0200F01D1022007E064
S3150800196CFFF7C0FE04E0012B15D0022B1AD002207B
S3150800197C30BB002835D11D4B1A6892B21C4B134448
S3150800198C5B0000221A6030221A4B1A800622164B6C
S3150800199C1B681A7210BD0B2C01D00220E8E7FFF762
S315080019AC75FEE5E7012C03D0032C04D00220DFE7F3
S315080019BCFFF798FEDCE7FFF725FFD9E70220D7E704
S315080019CC0D4B1B685B69204698470328D1D1092221
S315080019DCDDE70822DBE70822D9E70822D7E7082241
S315080019ECD5E70822D3E700BF60070020505C00400B
S315080019FC023000206807002038070020054B1B68BA
S31508001A0C5A8A10B10868104470478888801A188258
S31508001A1C002070476007002008B50C4B93F82C1073
S31508001A2C002000F047FB0A4B1B68187A082804D0DC
S31508001A3C092814BF0020012008BD4FF48052054B1D
S31508001A4C1A801022044B1A80F2E700BF700000209F
S31508001A5C60070020660700206807002070B51B4B3E
S31508001A6C1A6892B21A4B13445B001B88194A1268FF
S31508001A7C117A09291BD05B0003F1804303F5C04397
S31508001A8C5D1C19781170134C22685B7853702668A4
S31508001A9CB5F8030000F040FB70802668B5F807001F
S31508001AAC00F03AFBB0802368B5F80B20DA80094BB6
S31508001ABC1B6801221A72DB8823B1FFF75FFCFFF75C
S31508001ACCABFF70BDFFF70EFFF9E700BF505C004097
S31508001ADC043000206007002008B5124B1B681B7ADF
S31508001AEC022B1AD0042B1AD0032B0AD0052B08D09C
S31508001AFC072B0CD008220B4B1B681A72FFF78CFFAE
S31508001B0C08BDFFF74FFD074B1B681A7AF3E7064B20
S31508001B1C1B68DB6898470822EDE70822EBE70822E2
S31508001B2CE9E700BF600700203807002030B40F4BE8
S31508001B3C1D78002111E0CCB2A20002F1804202F518
S31508001B4CB842136823F0F0031B051B0D43F400433E
S31508001B5C43F08003234313600131A942EBD340F0D1
S31508001B6C8000034B186030BC704700BFA0000020F3
S31508001B7C4C5C004008B5154B1A68137A022B0AD030
S31508001B8C042B08D0062B0CD00822104B1B681A7293
S31508001B9CFFF742FF08BDFFF799FB0C4B1B681A7A37
S31508001BACF3E75378052B05D0094B1B689B689847B8
S31508001BBC0822EAE7137813F07F0FF5D1D078FFF7F0
S31508001BCCB5FF044B1B681B6A9847EDE760070020B6
S31508001BDC380700205C0700207047000008B5074B43
S31508001BEC074A136002221A72064B074A1360074902
S31508001BFC074A11601B68984708BD00BF40070020BC
S31508001C0C600700207000002038070020CC00002058
S31508001C1C5C07002010B582B00023ADF806307EE0D4
S31508001C2C1446136823F4E14323F070031B041B0CBE
S31508001C3C1360FFF79FFF236823F4804323F04003C8
S31508001C4C1B041B0C844A128812F4805F01D083F49F
S31508001C5C8053814A128812F4005F01D083F4005332
S31508001C6C7E4A128812F0100F01D083F010037B4ABB
S31508001C7C128812F0200F01D083F020039BB243F494
S31508001C8C004343F08003764A136002B010BD744CCF
S31508001C9C236823F070031B051B0D2360FFF7DEFE7C
S31508001CAC236823F4804323F040031B041B0C6A4A65
S31508001CBC128812F4805F01D083F48053664A128826
S31508001CCC12F4005F01D083F40053644A128812F0B0
S31508001CDC100F01D083F01003604A128812F0200FFF
S31508001CEC01D083F020039BB243F4004343F08003F6
S31508001CFC5B4A1360C9E79B0003F1804303F5B843BD
S31508001D0C1A6892B2ADF80620BDF8062012F4004FF8
S31508001D1C7DD1BDF8063013F0800F40F08680514B0C
S31508001D2C1B6899B2504A118013F4004FADD04E4B34
S31508001D3C1B8803F00F034D4A1370002BDBD1484A5E
S31508001D4C116889B2444B1980198801F0300143484F
S31508001D5C0180198801F440511980136823F48043D3
S31508001D6C23F040031B041B0C83F4005383F020035D
S31508001D7C43F4004343F0800313603B4B1B8813F07A
S31508001D8C100F3FF44DAF364B1B689BB2ADF80630BF
S31508001D9CBDF8063013F4006F7FF479AFBDF8063042
S31508001DAC13F4004FBBD02E4C236823F070031B058D
S31508001DBC1B0D2360FFF790FE236823F4804323F062
S31508001DCC40031B041B0C244A128812F4805F01D0B2
S31508001DDC83F48053204A128812F4005F01D083F4EE
S31508001DEC00531E4A128812F0100F01D083F010030C
S31508001DFC1A4A128812F0200F01D083F020039BB2E6
S31508001E0C43F4004343F08003154A13603DE71A6810
S31508001E1C22F070021205120D1A60144B1B78013B46
S31508001E2C134A52F82330984773E710490B789B00EE
S31508001E3C03F1804303F5B8431A6822F4E14222F011
S31508001E4C70021204120C1A600B78013B094A52F8FC
S31508001E5C2330984763E700BF660700206807002011
S31508001E6C005C0040445C00406A0700203C070020E8
S31508001E7C3C000020200000200132521001F10051D4
S31508001E8C01F54051490062B110B40378447843EA2D
S31508001E9C042321F8043B0230013A002AF5D110BC80
S31508001EAC704770470132521001F1005101F540514B
S31508001EBC490004E00B6820F8023B013A0431002A79
S31508001ECCF8D1704720F0070080B2014B18607047B4
S31508001EDC505C0040800000F1804000F5B840036873
S31508001EEC1BB223F4EC4323F07003194389B2016047
S31508001EFC7047800000F1804000F5B84003689BB23B
S31508001F0C23F4E04323F040039BB211F0100F01D0E9
S31508001F1C83F0100311F0200F01D083F0200343F453
S31508001F2C004343F0800303607047800000F1804053
S31508001F3C00F5B84003689BB223F4804323F0700382
S31508001F4C9BB211F4805F01D083F4805311F4005FC7
S31508001F5C01D083F4005343F4004343F08003036039
S31508001F6C7047800000F1804000F5B84003689BB2CA
S31508001F7C23F4E04323F0400383F0300343F4004397
S31508001F8C43F0800303607047800000F1804000F541
S31508001F9CB84003689BB223F4804323F0700383F4A0
S31508001FAC405343F4004343F08003036070478000BA
S31508001FBC00F1804000F5B84003681BB223F4F873AF
S31508001FCC1B051B0D43F4004343F080030360704765
S31508001FDC800000F1804000F5B840036813F4804F88
S31508001FEC09D0036823F0F0031B051B0D43F440438B
S31508001FFC43F0800303607047800000F1804000F5D1
S3150800200CB840036813F0400F09D0036823F0F003B7
S3150800201C1B051B0D43F4004343F0C00303607047D4
S3150800202C064B1B689BB203EBC00000F1005000F591
S3150800203C405040004908490001607047505C004018
S3150800204C054B1B689BB203EBC000044B03445B00B7
S3150800205C4908490019607047505C0040043000205C
S3150800206C054B1B689BB203EBC00000F1005000F552
S3150800207C4050400000887047505C0040044B1B6879
S3150800208C9BB203EBC000034B03445B0018887047F4
S3150800209C505C004004300020044B1B689BB203EBD9
S315080020ACC000034B03445B0019607047505C00404A
S315080020BC023000200E4B1B689BB203EBC0000D4B85
S315080020CC03445B003E290AD94A0911F01F0F01D1B6
S315080020DC013A92B2920242F400421A6070474A08D8
S315080020EC11F0010F00D0013292021A60704700BF3E
S315080020FC505C004006300020054B1B689BB203EB76
S3150800210CC000044B03445B001888C0F309007047F1
S3150800211C505C004006300020C3B2000A40EA032097
S3150800212C704700000020044B18604FF40643034A1E
S3150800213C1380034A13607047445C00406407002010
S3150800214C405C004070B50E4600F07F052846FFF748
S3150800215CD3FF04462846FFF791FF22460146304630
S3150800216CFFF7A0FE204670BD00B583B0002301938F
S3150800217C009303F1804303F504331A6842F0010215
S3150800218C1A605968414A0A405A601A6822F08472E1
S3150800219C22F480321A601A6822F480221A605A686D
S315080021AC22F4FE025A604FF41F029A601A6842F42F
S315080021BC80321A60364B1B6803F400330093019B7C
S315080021CC01330193009B23B9019A40F2DC539A42DE
S315080021DCF0D12F4B1B6813F4003F51D02D4B1A68C6
S315080021EC42F010021A601A6822F003021A601A6882
S315080021FC42F002021A60A3F580535A685A605A686C
S3150800220C42F400525A605A6842F480625A605A681C
S3150800221C22F47C125A605A6842F4E8125A601A6818
S3150800222C42F080721A601A4B1B6813F0007FFAD0C2
S3150800223C174B5A6822F003025A605A6842F0020297
S3150800224C5A60134B5B6803F00C03082BF9D1104B3F
S3150800225C9A6942F004029A610F4A116821F00F013B
S3150800226C1160116841F0040111605A6822F4800269
S3150800227C5A60DA6942F40002DA6103B05DF804FBCD
S3150800228C67210648FEF744FCA8E700BF0000FFF8E4
S3150800229C001002400020024000080140D026000829
S315080022AC08B5FFF761FFFEF763FCFEF76FFCFCE76A
S315080022BCDFF834D0002103E00C4B5B584350043153
S315080022CC0B480C4B42189A42F6D30B4A02E00023F1
S315080022DC42F8043B094B9A42F9D3FEF74BFF00F040
S315080022EC55F9FFF7DDFF7047005000208C270008D2
S315080022FC00000020F0000020F00000206C070020F1
S3150800230CFEE708B5FEF78CFB08BD08B5FEF7C2FB61
S3150800231C08BD000008B5044B1B68052B00D008BD8A
S3150800232CFEF77EFBFBE700BF2C07002008B51A4B0F
S3150800233C1B689BB2194A13801388194A128803F42E
S3150800234C00731A4210D1154B1B88154A128803F4D0
S3150800235C00431A4214D1114B1B88114A128803F4F4
S3150800236C80631A420FD108BD4FF6FF520A4B1A600A
S3150800237C0C4A13780133DBB21370FFF7CBFFE2E795
S3150800238CFFF748FCE7E74FF6FF32034B1A60064B9C
S3150800239C5B689847E7E700BF445C00406A07002083
S315080023AC640700202A07002070000020034B9B7A44
S315080023BC13B10522024B1A60704700BF4007002074
S315080023CC2C0700200422014B1A6070472C070020AA
S315080023DC7047704706280BD00023EBB110B50F4A8F
S315080023EC126893610024548220469847204610BDF3
S315080023FC0A4B1A68137803F07F03012B01D00023CC
S3150800240CEBE7537923B99378212B03D00023E4E720
S3150800241C0023E2E7024BE0E7022070476007002042
S3150800242C592500080220704709B10220704708B1E7
S3150800243C022070470020704710B5FEF74FFB054B7E
S3150800244C1B6800249C7200F089F8FFF76BFE024BA0
S3150800245C1C6010BD600700202C07002010B5264B09
S3150800246C1B6800249C72254AD2795A72DC72204663
S3150800247CFFF728FD4FF400712046FFF72BFD1021BE
S3150800248C2046FFF736FD40212046FFF7D9FD80216F
S3150800249C2046FFF7C5FD2046FFF789FD184B93F834
S315080024AC2C102046FFF706FE2046FFF76DFD214649
S315080024BC0120FFF70FFD4FF480710120FFF7B0FDE7
S315080024CCC0210120FFF7BCFD40210120FFF7E4FDE8
S315080024DC40210120FFF7EEFD4FF440510120FFF794
S315080024EC24FD20210120FFF704FD2046FFF71EFBE3
S315080024FC0122044B1A6010BD60070020DC26000878
S3150800250C700000202C07002008B50249FFF776FA60
S3150800251C08BD00BF6800002008B50249FFF76EFA2F
S3150800252C08BD00BF6000002008B5064B1B68DB78A9
S3150800253C052B05D8044901EBC301FFF75FFA08BD63
S3150800254C002008BD60070020A400002008B5024939
S3150800255CFFF754FA08BD00BF5800002008B5012043
S3150800256CFEF770FD064B01221A6000201860054A1A
S3150800257C10604FF4E05204490A801A6008BD00BF87
S3150800258C405C0040445C00406407002070B50025A0
S3150800259C0C4E0D4CA41BA410A54209D100F01AF838
S315080025AC00250A4E0A4CA41BA410A54205D170BDE1
S315080025BC56F8253098470135EEE756F825309847F2
S315080025CC0135F2E7842700088427000884270008C9
S315080025DC88270008F8B500BFF8BC08BC9E467047AB
S311080025ECF8B500BFF8BC08BC9E46704756
S315080025F800400008002000000200000000600008F3
S3150800260800200000030000000080000800200000E9
S315080026180400000000A000080020000005000000D3
S3150800262800C00008002000000600000000E00008BE
S315080026380020000007000000000001080020000034
S31508002648080000000020010800200000090000001A
S3150800265800400108002000000A0000000060010888
S31508002668002000000B000000008001080020000080
S315080026780C00000000A00108002000000D00000062
S3150800268800C00108002000000E00000000E0010854
S31508002698002000000F0000002E2E2F2E2E2F2E2E83
S315080026A82F2E2E2F536F757263652F41524D434D4A
S315080026B8335F53544D333246312F7573622E630098
S315080026C84F70656E424C54002E2E2F6D61696E2E22
S315080026D86300000009022000010100C03209040055
S315080026E80002FF00000407058102400000070501F3
S315080026F8024000001201100100000040501DAC60A5
S3150800270800010102030100002C03570069006E004E
S315080027185500530042002000420075006C006B000B
S31508002728200049006E0074006500720066006100AA
S3150800273863006500040309042603570069006E0050
S315080027485500530042002000420075006C006B00DB
S3150800275820004400650076006900630065000000F3
S315080027681A034F00700065006E0042004C005400C2
S3110800277820005500730065007200000088
S309080027843101000809
S309080027880D01000829
S3150800278C040000001C0353004500520031003200BF
S3150800279C3300340035003600370038003900300075
S315080027AC0F230008E51B0008E51B0008E51B0008BD
S315080027BCE51B0008E51B0008E51B000817230008A5
S315080027CCE51B0008E51B0008E51B0008E51B0008CF
S315080027DCE51B0008E51B0008EE26000809000000AA
S315080027ECDC26000820000000FC2600081200000069
S315080027FC4524000869240008DD230008DF230008A7
S3150800280CE1230008312400083524000815250008A2
S3150800281C25250008352500080000000040000000AA
S3150800282C030100003C270008040000006827000884
S3150800283C1A000000402700082600000004000020AB
S3150800284C1C000000102700082C000000E51B0008DF
S3150800285CB9230008E51B0008E51B0008E51B000862
S3150800286CE51B0008E51B0008E51B0008D12300083A
S705080022BD13
